:0410000061EF08F0A4
:101018002180D8CF05F0E8CF06F0E0CF07F0FACF6F
:1010280008F0FBCF09F0E9CF0AF0EACF0BF0E1CFE7
:101038000CF0E2CF0DF0D9CF0EF0DACF0FF0F3CFEE
:1010480010F0F4CF11F0F6CF12F0F7CF13F0F8CF7D
:1010580014F0F5CF15F0F2A00CD08C70F290010EC0
:10106800016E000E026E000E036E000E046E82EC1E
:1010780009F015C0F5FF14C0F8FF13C0F7FF12C040
:10108800F6FF11C0F4FF10C0F3FF0FC0DAFF0EC067
:10109800D9FF0DC0E2FF0CC0E1FF0BC0EAFF0AC098
:1010A800E9FF09C0FBFF08C0FAFF07C0E0FF06C060
:1010B800E8FF05C0D8FF2190100098EF09F0000064
:1010C8000000000000005F00000007000700147F18
:1010D800147F14242A7F2A12231308646236495580
:1010E80022500005030000001C2241000041221C80
:1010F8000014083E081408083E0808005030000094
:101108000808080808006060000020100804023E73
:101118005149453E00427F400042615149462141C4
:10112800454B311814127F1027454545393C4A492B
:1011380049300171090503364949493606494929A3
:101148001E00363600000056360000081422410002
:10115800141414141400412214080201510906320F
:101168004979413E7E1111117E7F494949363E41F8
:101178004141227F4141221C7F494949417F090958
:1011880009013E4149497A7F0808087F00417F41AB
:10119800002040413F017F081422417F40404040E9
:1011A8007F020C027F7F0408107F3E4141413E7F51
:1011B800090909063E4151215E7F09192946464918
:1011C80049493101017F01013F4040403F1F204014
:1011D800201F3F4038403F63140814630708700815
:1011E800076151494543007F41410002040810202E
:1011F8000041417F00040201020440404040400099
:101208000102040020545454787F48444438384438
:10121800444420384444487F3854545418087E09BC
:1012280001020C5252523E7F0804047800447D406B
:10123800002040443D007F1028440000417F4000CA
:101248007C041804787C0804047838444444387CC6
:1012580014141408081414187C7C0804040848544E
:10126800545420043F4440203C4040207C1C2040F3
:10127800201C3C4030403C44281028440C5050501E
:101288003C4464544C44000836410000007F000090
:1012980000413608001008081008784641467800D2
:1012A80095909380000EC26EC180C182C184C186B0
:1012B800F28EF286F19EF18CF190010E166E000E00
:1012C800176E000E186E000E196E6CEC09F0F5D74B
:1012D80003D0040EE82EFED7FF0E1626FF0E1722A7
:1012E800FF0E1822FF0E19221628F3E11728F1E144
:1012F8001828EFE11928D8B41200EBD703D0040E50
:10130800E82EFED7FF0E0126FF0E0222FF0E032253
:10131800FF0E04220128F3E10228F1E10328EFE19E
:101328000428D8B41200EBD700EE1AF0070EEE6AC4
:10133800E806FDE121902192000EF86E000154EFBD
:0213480009F0AA
:020000040020DA
:08000000FFFFFFFFFFFFFFFF00
:020000040030CA
:0E000000240E3F1EFF8181FF0FC00FE00F4056
:00000001FF
